:020000040000FA
:100000008316031306309F00003085000030860001
:10001000003087000030880003308900831203130A
:100020005030A000F001F101F201F301F401F901F7
:100030008701FE0186118601861683120317FF30A1
:100040008D0083120313B920FD008030F500472195
:10005000FF30F800D320F920B621F030F800D3208B
:10006000F920B6210330F800D320F920B621ED3075
:10007000F800D320F920B6210730F800D320F9206A
:10008000B621ED30F800D320F920B6210030F80079
:10009000D320F920B621FA30F800D320F920B62178
:1000A0007D08003A031958287D08013A031D7D2870
:1000B00083160313FF30870083120313F830F80010
:1000C000D320F920B621ED30F800D320F920B62155
:1000D0000230F800D320F920B621FF30F500472187
:1000E000ED30F800D320F920B6210030F800D320FD
:1000F000F9208030F5004721B8287D08023A031D19
:100100009B28ED30F800D320F920B6210430F80008
:10011000D320F920B621FF30F5004721ED30F8005B
:10012000D320F920B6210030F800D320F920803008
:10013000F5004721B8287D08033A031DB828ED30A3
:10014000F800D320F920B6210130F800D320F9209F
:10015000B621FF30F5004721ED30F800D320F9201B
:10016000B6210030F800D320F9208030F500472177
:10017000492A831603178C130C14831203170C08D7
:10018000831203130800831603178C130C158B13AB
:1001900055308D00AA308D008C148B1783120313F9
:1001A000B621B6210800FC01FB007B18FC0AFB18F5
:1001B000FC0A7B19FC0AFB19FC0A7B1AFC0AFB1AD5
:1001C000FC0A7B1BFC0AFB1BFC0A7C08013A031996
:1001D000F7287C08033A0319F7287C08053A031925
:1001E000F7287C08073A0319F7282114F82821106A
:1001F00008008316031300308900831203130914C7
:1002000089105521831603130230890083120313CA
:100210000910552189180A29781C09107818091421
:100220004221F81C0910F81809144221781D091000
:10023000781909144221F81D0910F81909144221EE
:10024000781E0910781A09144221F81E0910F81AAC
:1002500009144221781F0910781B09144221F81F44
:100260000910F81B09144221211C09102118091436
:1002700042210914831603130330890083120313E8
:1002800055210800891C4229891844290800FA30A0
:10029000F700000000000000000000000000000067
:1002A000F70B4929F50B47290034A008F500000099
:1002B000000000000000000000000000F50B5729BE
:1002C00008001822F81FB621F81BC0211822781F39
:1002D000B621781BC0211822F81EB621F81AC021B9
:1002E0001822781EB621781AC0211822F81DB621CE
:1002F000F819C0211822781DB6217819C0211822BA
:10030000F81CB621F818C021EB211822F81FB621DD
:10031000F81BC0211822781FB621781BC021182293
:10032000F81EB621F81AC0211822781EB621781AB4
:10033000C0211822F81DB621F819C0211822781DF5
:10034000B6217819C0211822F81CB621F818C0214E
:10035000EB210F308A00A12F0000000000341B3079
:10036000F50000000000F50BB12900342030F60044
:10037000C130F5000000F50BBA29F60BB82900349E
:10038000000000000000000000000000000000006D
:10039000000000000000000000000000000000005D
:1003A00000000000000000002030F6006C30F50076
:1003B0000000000000000000000000000000F50B3D
:1003C000D82900000000000000000000000000002C
:1003D000F60BD629003418221E30F500000000006C
:1003E0000000F50BEE293030F600F530F500000086
:1003F00000000000F50BF729F60BF5290034182250
:100400002E30F500000000000000F50B022A00006D
:1004100000000000F50B072A4030F600F630F5002A
:10042000000000000000F50B102AF60B0E2A003425
:1004300086150000AC2100008611AF218615000052
:10044000AC2100008611AF2186150000AC21000010
:100450008611AF2186150000AC2100008611AF2166
:1004600086150000AC2100008611AF218615000022
:10047000AC21000086110034ED30F800D320F920C3
:10048000B6217908F800D320F920B6210F308A0070
:10049000A82F9222701B692A7D08003A031D532A57
:1004A00018308A0000287D08013A031D5A2A1830A6
:1004B0008A0000287D08023A031D612A0F308A0055
:1004C000862F7D08033A031D682A0F308A00A92F62
:1004D000492AF01F4C2AFA017208703A0319882A37
:1004E000FA0A7208693A0319882AFA0A7208723AF3
:1004F0000319882AFA0A72087A3A0319882A7208B4
:100500006B3A0319882A7208733A0319882A4C2A0D
:100510007A08831203178C00FF308D0083120313B7
:10052000C3200028F201F301F4010909033903197A
:10053000922A9E2208308A0000280800831603139E
:10054000033089008312031389180918A42A891C0F
:100550000918A72A091808002A23091C731009186A
:1005600073142A23091CF3100918F3142A23091CF5
:100570007311091873152A23091CF3110918F315AF
:100580002A23091C7312091873162A23091CF31253
:100590000918F3162A23091C7313091873172A2341
:1005A000091CF3130918F3172A232A237308833A23
:1005B000031900287308013A031900287308F03A58
:1005C0000319ED2A7308F200831603130030890023
:1005D0008312031309148910080089180918ED2AD9
:1005E000891C0918F02A091808002A23091C74100C
:1005F000091874142A23091CF4100918F4142A2366
:10060000091C7411091874152A23091CF4110918FE
:10061000F4152A23091C7412091874162A23091CBC
:10062000F4120918F4162A23091C741309187417F4
:100630002A23091CF4130918F4172A232A237408FF
:10064000F200831603130030890083120313091488
:0E06500089100800891C2A2B89182C2B080001
:10100000701C0528F01C08280A28F01C0A2808284B
:10101000F1170B28F1137308F03A031D5F287208CB
:10102000143A0319EA2F7208123A03194A2872086F
:10103000593A03194C287208113A03194F287208BB
:10104000583A031951287208193A0319532872089B
:10105000393A031955287208763A03195728720845
:101060005F3A0319582872088B3A031959287208F5
:101070008C3A03195B288D3A03195D287D08013AE3
:10108000031D49288713831603137F3087008312BB
:101090000313EA2FF010EA2FF0107011EA2FF0116D
:1010A000EA2F7012EA2FF012EA2F7013EA2FEA2FBC
:1010B000EA2FF110EA2F7111EA2FF111EA2F7208CD
:1010C000143A031990287208123A03199A287208E0
:1010D000593A03199C287208113A03199F2872087B
:1010E000583A0319A1287208193A0319A32872085B
:1010F000393A0319A5287208763A0319A728720805
:101100005F3A0319B32872088B3A0319BD28720895
:101110008C3A0319BF2872088D3A0319C128E72FAA
:10112000701C962870107911A527EA2F7014791574
:10113000A527EA2FF014EA2F7015F014EA2FF01506
:10114000EA2F7016EA2FF016EA2F7017EA2FF01F19
:10115000AE28F0138616F910A527EA2FF01786128D
:10116000F914A527EA2F711CB92871107910A52749
:10117000EA2F71147914A527EA2FF114EA2F7115BB
:10118000EA2FF115EA2F7208773A031DCE28F11FD6
:10119000D630F11BD630F8009E27A22F72087E3A77
:1011A000031DD928F11F5830F11B5830F8009E2735
:1011B000A22F7208843A031DE428F11FD030F11BDE
:1011C000D030F8009E27A22F72087C3A031DEF282A
:1011D000F11F9630F11B9630F8009E27A22F72085F
:1011E000713A031DFA28F11FD230F11BD230F800FA
:1011F0009E27A22F7208703A031D0529F11FD430D3
:10120000F11BD430F8009E27A22F7208693A031D03
:101210001029F11FAE30F11BAE30F8009E27A22F2F
:101220007208723A031D1B29F11FA030F11BA03078
:10123000F8009E27A22F72087A3A031D2629F11F73
:10124000A830F11BA830F8009E27A22F72086B3A35
:10125000031D3129F11FA630F11BA630F8009E278F
:10126000A22F7208733A031D3C29F11FA430F11B11
:10127000A430F8009E27A22F7208743A031D482953
:10128000701CF11FAA30F11BAA30F8009E27A22F74
:1012900072086C3A031D5329F11FAC30F11BAC30BE
:1012A000F8009E27A22F7208753A031D5E29F11FD0
:1012B000A230F11BA230F8009E27A22F72087D3ABF
:1012C000031D8C2FF11FDC30F11BDC30F8009E2752
:1012D000A22F7208153A031D7429F11F5430F11B17
:1012E0005430F8009E27A22F7208133A031D7F295D
:1012F000F11F6630F11B6630F8009E27A22F72089E
:101300005B3A031D892FF11F6830F11B6830F8002C
:101310009E27A22F7208773A031D9529F11FD63018
:10132000F11BD630F8009E27E42F72087E3A031D89
:10133000A029F11F5830F11B5830F8009E27E42FE8
:101340007208843A031DAB29F11FD030F11BD03055
:10135000F8009E27E42F72087C3A031DB629F11F7E
:101360009630F11B9630F8009E27E42F7208713AF0
:10137000031DC129F11FD230F11BD230F8009E2786
:10138000E42F7208703A031DCC29F11FD430F11BF1
:10139000D430F8009E27E42F7208693A031DD7293C
:1013A000F11FAE30F11BAE30F8009E27E42F72081B
:1013B000723A031DE229F11FA030F11BA030F800A2
:1013C0009E27E42F72087A3A031DEE29701CF11F44
:1013D000A830F11BA830F8009E27E42F72086B3A62
:1013E000031DF929F11FA630F11BA630F8009E2736
:1013F000E42F7208733A031D042AF11FA430F11B75
:10140000A430F8009E27E42F7208743A031D0F2AB7
:10141000F11FAA30F11BAA30F8009E27E42F7208B2
:101420006C3A031D1A2AF11FAC30F11BAC30F800E6
:101430009E27E42F7208753A031D252AF11FA2305A
:10144000F11BA230F8009E27E42F72087D3A031D9D
:10145000AF2FF11FDC30F11BDC30F8009E27E42FAA
:101460007208153A031D552A701C4E2AF11F3A2A9C
:10147000F11B442ACE30F8009E275430F8009E27F6
:10148000CE30F8009E27E42FCE30F8009E2754304F
:10149000F8009E27CE30F8009E27E42FF11F54302D
:1014A000F11B5430F8009E27E42F7208133A031DF5
:1014B0007C2A701C742AF11F5F2AF11B692ACE3026
:1014C000F8009E27E630F8009E27CE30F8009E27D1
:1014D000E42FCE30F8009E27E630F8009E27CE306D
:1014E000F8009E27D127E42FF11F6630F11B6630EC
:1014F000F8009E27D127E42F72085B3A031DAC2F1A
:10150000701C892AF11F6830F11B6830F8009E2793
:10151000E42FF11F6830F11B6830F8009E27E42F9C
:10152000F11F942AF11B9F2ACE30F8009E27E83045
:10153000F8009E27CE30F8009E27D127E42FCE302A
:10154000F8009E27E830F8009E27CE30F8009E274E
:10155000D127E42FF11FAE2AF11BB92ACE30F800B3
:101560009E276230F8009E27CE30F8009E27D127B4
:10157000E42FCE30F8009E276230F8009E27CE3050
:10158000F8009E27D127E42FF11FC82AF11BD32A88
:10159000CE30F8009E276630F8009E27CE30F80047
:1015A0009E27D127E42FCE30F8009E276630F80022
:1015B0009E27CE30F8009E27D127E42FF11FE22A84
:1015C000F11BED2ACE30F8009E276830F8009E27E8
:1015D000CE30F8009E27D127E42FCE30F8009E278A
:1015E0006830F8009E27CE30F8009E27D127E42FE0
:1018000082070034003400340034003400340034E3
:10181000BE3498340034003400340034EA34E83400
:10182000B034003400340034523400348E34AE34DA
:10183000B83400340034F034C834C0348034A034B8
:10184000B6340034F634F834C6348834A634A834B8
:10185000B4340034E234F434C43484348634A434EC
:10186000BA340034FC34FA34CC34CA348A34AA345E
:101870003E3400340034F234C2348C34AC34A234FC
:1018800030340034D23492348234EC34D434DC3406
:1018900038340034DA34D0349A34EA34E434EA3474
:1018A000363400340034EA342834EA34EA34343448
:1018B000EA3400340034FE349634283400343A34A8
:1018C0000034EE34E034B2349E349434BC34983472
:1018D0009C340034BC34DE34E0349034EA34903448
:1018E000EA349C349434EE34EA34DE349E340034EA
:1018F000D6340034FE34EA3400349634EA345834B2
:0C19000000340034003400340034D034D3
:101A000082070034003400340034003400340034E1
:101A1000BE3418340034003400340034EA341C344A
:101A2000B0340034003400345A3400340E342E34D0
:101A3000B834003400347034483440340034203436
:101A4000B634003476347834463408342634EA34F4
:101A5000B4340034623474344434043406342434EA
:101A6000BA3400347C347A344C344A340A342A345C
:101A70003E3400340034723442340C34D6342234D0
:101A8000303400341634123402346C3450345C3444
:101A900038340034D834E6341A34EA3464345634F2
:101AA000363400340034EA342C34EA34EA34343442
:101AB000EA3400340034FE3458342C3400343A34E0
:101AC00000346E34603432341E3414343C341834F0
:101AD0009C3400343C345E34E0341034EA34103446
:101AE000EA349C349434EE34EA34DE349E340034E8
:101AF000D6340034FE34EA3400349634EA345834B0
:0C1B000000340034003400340034D034D1
:101C000082070034003400340034003400340034DF
:101C1000BE3418340034003400340034EA341C3448
:101C2000B0340034003400345A3400340E342E34CE
:101C3000B834003400347034483440340034203434
:101C4000B634003476347834463408342634EA34F2
:101C5000B4340034623474344434043406342434E8
:101C6000BA3400347C347A344C344A340A342A345A
:101C70003E3400340034723442340C34D6342234CE
:101C8000303400341634123402346C3450345C3442
:101C900038340034D834E6341A34033464345634D7
:101CA00036340034003405342C340734EA34343408
:101CB000EA3400340034FE3458342C3400343A34DE
:101CC00000346E34603432341E3414343C341834EE
:101CD0009C3400343C345E34E0341034EA34103444
:101CE000EA349C349434EE34EA34DE349E340034E6
:101CF000D6340034FE34EA3400349634EA345834AE
:0C1D000000340034003400340034D034CF
:101E000082070034003400340034003400340034DD
:101E1000BE3498340034003400340034EA34E834FA
:101E2000B034003400340034523400348E34AE34D4
:101E3000B83400340034F034C834C0348034A034B2
:101E4000B6340034F634F834C6348834A634A834B2
:101E5000B4340034E234F434C43484348634A434E6
:101E6000BA340034FC34FA34CC34CA348A34AA3458
:101E70003E3400340034F234C2348C34AC34A234F6
:101E800030340034D23492348234EC34D434DC3400
:101E900038340034DA34D0349A34EA34E434013457
:101EA000363400340034EA342834EA34EA34343442
:101EB000EA3400340034FE349634283400343A34A2
:101EC0000034EE34E034B2349E349434BC3498346C
:101ED0009C340034BC34DE34E0349034EA34903442
:101EE000EA349C349434EE34EA34DE349E340034E4
:101EF000D6340034FE34EA3400349634EA345834AC
:101F000000340034003400340034D034F01E892F03
:101F10006929F01F8C2FC328F11F932F0D308A00E1
:101F200072080025982F0C308A0072080024982F20
:101F3000F800EA3A03199D2F9E27A22F01308A004C
:101F40006129080002308A00612A02308A003C2A96
:101F50000800F01EAC2F302AF01FAF2F8A29F11F86
:101F6000B62F0E308A0072080025BA2F0F308A0073
:101F700072080025F800013A0319902A7808F80041
:101F8000053A0319AA2A7808033A0319C42A7808DB
:101F9000073A0319DE2A7808EA3A0319D02F9E2758
:101FA000E42F8230F500000000000000F50BD32F75
:101FB0003030F600F530F500000000000000F50BB1
:101FC000DC2FF60BDA2F003402308A00682A023048
:101FD0008A009D2A7D08013A031DEF2F87130230E6
:041FE0008A00922AB7
:10300000831203137208643A031D0A28F01D0A286C
:10301000F01A8E2018308A003F205F206720712030
:103020007E08FD3A03198C287E08FE3A031993287E
:103030007E08FA3A031907297E088F3C03182428D2
:103040007E08BF3C031897287E08870003193C2898
:1030500083160313003087008312031387177D083C
:10306000003A031D3C2801306021871383160313A7
:103070007F3087008312031319308A007029720889
:10308000843A031D45287B30F20072087F3C031C04
:103090005D281A308A0072080022FE00711C0800A8
:1030A0007E08033A1B3003195B287E080F3A09306B
:1030B00003195B287E08FE000800FE010800F11FCE
:1030C00008001A308A0072088022FE000800F019F9
:1030D0006B28701E08001B308A0072080023FE0057
:1030E0000800F01A7528701F0800F019031D7D28CC
:1030F0007208643A031D7D288C281B308A007208F0
:103100008023FE0008007208870083160313003036
:103110008700831203133C288E206D2906150000BA
:1031200000000611080006165F2106123C28711CDB
:10313000A6287E089B3C031CA0282430FE07A62856
:103140007E08B33C0318A6282430FE027E08CA205D
:103150001030FA00E520FA007A0A031DB228203068
:103160006021C7287A0887000319C928831603132A
:10317000003087008312031387175F218713043001
:10318000602183160313FF30870083120313FA0BA9
:10319000AA283C28FA00831203171D308F00003044
:1031A0008D00831203139030FA020319E228831270
:1031B000031710308D07031CDE288F0A83120313B8
:1031C000FA0BD728831203130800831603178C17F2
:1031D0000C14000000000000831203178D0A0C0875
:1031E000831203130800831603178C170C158B1317
:1031F00055308D00AA308D008C14000000000000B6
:103200008B17831203178D0A8312031308000730EC
:103210005821FE0102308A00922218308A003F2095
:103220005F20672071207E088F3C03186D297E087F
:10323000BF3C031C6D29053058217E08CA20103080
:10324000FA0002308A00922219308A000130582197
:103250007208623A031D2F29FF30FE0040293F20EB
:103260005F20672071207E087F3C031CFE017E08E2
:103270008700831603130030870083120313871718
:10328000831203177E088C008E01F3205F21053026
:103290005821871383160313FF308700831203130B
:1032A0007E0803195529FA0B2129003058216D2970
:1032B000F90002308A003C2219308A0008000230EE
:1032C000A5006521A50B612900347D30A400A30170
:1032D000A30B6829A40B6729003400308A0000285A
:0632E00002308A005A2AA8
:1034000082070034003400340034003400340034C7
:103410009034033400340034003400340F345E340C
:1034200091340034113412343C3414345134313476
:1034300092340034193459345334413457343234CB
:1034400093340034433458344434453434343334BE
:1034500094340034203456344634543452343534A1
:10346000953400344E344234483447345A34363478
:103470009634003439344D344A3455343734383482
:10348000973400342C344B3449344F34303439348D
:10349000983400342E342D344C345C3450347E3423
:1034A0009934003400345B3423345D343C349A3432
:1034B0001834583459340D342B34233400349B34AD
:1034C00000340A34083413340B34043404347F34A5
:1034D0000534003431340934343437340A34013497
:1034E0000B3430342C34323435343634383476348A
:1034F0002F3400340D3433342D342B3439342A3402
:1035000082070034003400340034003400340034C6
:103510009C341B3400340034003400340F346034E5
:103520009D340034113412343E3414347134213457
:103530009E3400341934793473346134773422344E
:103540009F34003463347834643465342434403434
:10355000A034003420347634663474347234253424
:10356000A13400346E346234683467347A342634DB
:10357000A234003439346D346A3475342F3428342D
:10358000A33400343B346B3469346F343D34293414
:10359000A43400343A345F346C347C3470343F34B7
:1035A000A534003400347B3427347D343E34A634D3
:1035B0000034583459340D342A3427340034A734B5
:1035C00000340A34083413340B345F3402347F344B
:1035D0000534003431340934343437340A340C348B
:1035E0000B3430342C343234353436343834763489
:1035F0002F3400340D3433342D342B343934023429
:1036000082070034003400340034003400340034C5
:10361000A834FE34003400340034003417345E34EF
:10362000A9340034113412343C34143411340134CC
:10363000AA340034193419341334013417340234E1
:10364000AB34003403341834043405340434033404
:10365000AC340034203416340634143412340534B7
:10366000AD3400340E340234083407341A340634CE
:10367000AE34003439340D340A3415340734083488
:10368000AF3400342C340B3409340F340034093493
:10369000B03400342E342D340C341C3410347E34C9
:1036A000B134003400341E3423341D343C34B2347D
:1036B0000034583459340D342B3427340034B334A7
:1036C00000340A34083413340B34133413341234F2
:1036D0000534003431340934343437340A34143482
:1036E0000B3430342C343234353436343834763488
:1036F0002F3400340D3433342D342B3439342A3400
:1037000082070034003400340034003400340034C4
:10371000B434FD3400340034003400340034003458
:10372000B5340034003400340034003460340034E4
:10373000B634003400340034003400340034003433
:10374000B734003400340034003400340034003422
:10375000B834003400340034003400340034003411
:10376000B934003400340034003400340034003400
:10377000BA340034003400340034003400340034EF
:10378000BB340034003400340034003400340034DE
:10379000BC340034003400340034003400340034CD
:1037A000BD34003400340034003400340034BE34FE
:1037B000FA34003400340D34003400340034BF34A3
:1037C00000340A34083413341A347F3400347F341C
:1037D0000034003431341534343437340A3401348D
:1037E0001A3430342C3432343534363438340034EE
:1037F0002F3400340D3433342D342B3439342A34FF
:103A0000230020004F002000310030003000300043
:103A100020000D0000000000000000000000000079
:103A20002300200057002000310031002000310029
:103A300020000D0000000000000000000000000059
:103A4000230020005700200031003100200030000A
:103A500020000D0000000000000000000000000039
:103A60001200000000000000000000000000000044
:103A70000000000000000000000000000000000046
:103A80001300000000000000000000000000000023
:103A90000000000000000000000000000000000026
:103AA0000C0000000000000000000000000000000A
:103AB0000000000000000000000000000000000006
:103AC00007000000000000000000000000000000EF
:103AD00000000000000000000000000000000000E6
:103AE0000E000000000000000000000000000000C8
:103AF00000000000000000000000000000000000C6
:103B000014000000000000000000000000000000A1
:103B100000000000000000000000000000000000A5
:103B200042005900450020000D0000000000000088
:103B30000000000000000000000000000000000085
:103B4000160000000000000000000000000000005F
:103B50000000000000000000000000000000000065
:103B6000170000000000000000000000000000003E
:103B70000000000000000000000000000000000045
:103B8000530068006900660074002B004600310095
:103B90000000000000000000000000000000000025
:103BA000530068006900660074002B004600320074
:103BB0000000000000000000000000000000000005
:103BC000530068006900660074002B004600330053
:103BD00000000000000000000000000000000000E5
:103BE000530068006900660074002B004600340032
:103BF00000000000000000000000000000000000C5
:103C0000530068006900660074002B004600350010
:103C100000000000000000000000000000000000A4
:103C2000530068006900660074002B0046003600EF
:103C30000000000000000000000000000000000084
:103C4000530068006900660074002B0046003700CE
:103C50000000000000000000000000000000000064
:103C6000530068006900660074002B0046003800AD
:103C70000000000000000000000000000000000044
:103C8000530068006900660074002B00460039008C
:103C90000000000000000000000000000000000024
:103CA000530068006900660074002B004600310074
:103CB00030000000000000000000000000000000D4
:103CC000530068006900660074002B004600310054
:103CD00031000000000000000000000000000000B3
:103CE000530068006900660074002B004600310034
:103CF0003200000000000000000000000000000092
:103D000053007400720067002B0046003100000071
:103D100000000000000000000000000000000000A3
:103D200053007400720067002B0046003200000050
:103D30000000000000000000000000000000000083
:103D400053007400720067002B004600330000002F
:103D50000000000000000000000000000000000063
:103D600053007400720067002B004600340000000E
:103D70000000000000000000000000000000000043
:103D800053007400720067002B00460035000000ED
:103D90000000000000000000000000000000000023
:103DA00053007400720067002B00460036000000CC
:103DB0000000000000000000000000000000000003
:103DC00053007400720067002B00460037000000AB
:103DD00000000000000000000000000000000000E3
:103DE00053007400720067002B004600380000008A
:103DF00000000000000000000000000000000000C3
:103E000053007400720067002B0046003900000068
:103E100000000000000000000000000000000000A2
:103E200053007400720067002B0046003100300020
:103E30000000000000000000000000000000000082
:103E400053007400720067002B00460031003100FF
:103E50000000000000000000000000000000000062
:103E600053007400720067002B00460031003200DE
:103E70000000000000000000000000000000000042
:103E800003006C0074002B004600310000000000AD
:103E90000000000000000000000000000000000022
:103EA0000500000074002B004600320000000000F6
:103EB0000000000000000000000000000000000002
:103EC0000400000074002B004600330000000000D6
:103ED00000000000000000000000000000000000E2
:103EE00041006C0074002B0046003400000000000C
:103EF00000000000000000000000000000000000C2
:103F00001300000074002B00460035000000000084
:103F100000000000000000000000000000000000A1
:103F20000100000074002B00460036000000000075
:103F30000000000000000000000000000000000081
:103F40000700000074002B0046003700000000004E
:103F50000000000000000000000000000000000061
:103F600041006C0074002B00460038000000000087
:103F70000000000000000000000000000000000041
:103F800044004900520020000D0000000000000025
:103F90000000000000000000000000000000000021
:103FA0004500780069007400200000000000000057
:103FB0000000000000000000000000000000000001
:103FC0004C004F004100440020002200220000006D
:103FD00000000000000000000000000000000000E1
:103FE0004300530041005600200022000000000062
:103FF00000000000000000000000000000000000C1
:02400E00723FFF
:0243FE000100BC
:00000001FF
